:1000000072C095C03EC293C092C096C090C08FC0CF
:100010008EC08DC08CC08BC03EC189C088C000001E
:1000200000000000000000000000000023456C9864
:10003000C9FF040714233764A0FFFFFFFFFFFFFF82
:10004000FFFFFFFFFF000000000000000000234052
:100050005F7AB4FFFFFFFFFFFF00140008140008E1
:100060000E140004080E14000305080E1400040802
:100070000A0E1114000305080A0E101400030508E7
:100080000A0E1012140008000E00080E0004080EDC
:10009000000305080E0004080E1100080E1100F3FD
:1000A000F404080E10121400080A0C0E0F1012149B
:1000B00000080EED14000203040500041400040EF1
:1000C0001400040810140004080F1114000305089C
:1000D0000A0E0004080A0E00EEEDECEB140E080404
:1000E0000004080E000011241FBECFEDCDBF20E09C
:1000F000A0E6B0E001C01D92A437B207E1F7E5E742
:10010000F0E085E5808781E0838312821182118689
:100110008BE0828788E58387E1E6F0E08DEF8783D7
:100120008EEF8583712C55245A94B6D0D2C168CFF6
:100130001BBC19BC18BC0895189525B7277E25BF90
:1001400029B7226029BF21E022BF019728F020E1D2
:1001500088952150E9F7F9CF089588EE93E0EDCF27
:10016000369A3699FECF95B180916000892708951F
:1001700080917400E3E8F0E080838183828383834D
:100180000895CF93C72D81E0870D8F73782E662D4C
:1001900090E091D16FEF8C2F90E0CF918CC1FF92C6
:1001A0000F931F93CF93DF93F82E06E710E0CEE76F
:1001B000D0E0F11005C0CE0176D1F801808304C0F3
:1001C000F8016081CE0177D121970F5F1F4FC337B0
:1001D000D10579F7DF91CF911F910F91FF9008958D
:1001E000D0DF81E0DCCF811101C0A2CF815090E04F
:1001F000FC01E25EFF4FE491EBBDFC01EE5CFF4FC2
:10020000E491E9BDFC01EA5BFF4F849188BD08954C
:100210000F931F93CF93C82F8B01CC2359F085E008
:10022000E2DFC8018ADF84DFC80187DFC80185DF1C
:10023000C150F3CFCF911F910F910895CF93DF93CA
:10024000D82F64E170E08AE0E3DF84EF91E075DFAE
:100250008D2F64E61CD1CAE06C2F19D1892F68EC70
:1002600070E0D6DF7ADF8D2F6C2F11D1D92F0FD10F
:10027000892F68EC70E0CCDF70DF68EC70E08D2FC8
:10028000C7DF6BDF64E170E08AE0C2DF84EF91E0FA
:10029000DF91CF9152CF18951092740087E790E0CC
:1002A00002D1853519F0612C9BDF11C0712C872D8F
:1002B00090E0F9D0682E8F3F19F080E070DF07C022
:1002C000872D21E0270D722E803488F3F6CF8091A0
:1002D0007E008111AB9890917F00409178008091D1
:1002E0007600882311F040E09AE19F5F80E06AE5A4
:1002F00070E0C42FD0E09923A9F09B012F5F3F4FFE
:10030000F9013197E491A82FB0E0A559BF4FAC0F88
:10031000BD1FEC93EE2319F0822F861BEFCF915077
:10032000B901E9CF840F80938100442319F091E053
:1003300090936B0080938200962D953F18F520E1F5
:100340002515B0F0209183002F3F31F411DFE3E851
:10035000F0E094E09E0F06C09F5F692E9817B8F3F7
:10036000612CF5CF80818F5F81939E13FBCF0AC0F4
:10037000FFDE80917600811104C0809177008111A9
:1003800001C0612C512C8FEF8DBD80E68CBDAB9AE6
:100390008FE384BB8BE187BB8CEE88BB81E083BF9E
:1003A00091EA9ABD80BF8BB780628BBF8AB78560A8
:1003B0008ABF85B7806285BF78948CE287B986EC66
:1003C00086B93699FECF8FEF809360008CE291E082
:1003D000B4DEC6DE33DFFACF112416B8A9DE87B348
:1003E0008C7E87BB80E051E041E020E030E0A8E077
:1003F000999B06C0F9013197F1F79AB795609ABFBA
:1004000096B39A27999B03C0511003C034C0911131
:1004100007C040E3451588F581112FC050E049E041
:10042000652D71E0623308F070E0760F572E5111A0
:1004300008C0811105C081E0911103C080E001C0B6
:1004400081E0999895B7977E906195BFA895942F74
:10045000987011F490E401C090E6916091BD95B759
:10046000946895BF9B7F95BF78948895F89491B5D3
:100470009F7B91BDBDCF9111D3CF8FED8DBF1FBE9F
:100480000BDF999A552011F0189501C0A5DF991B33
:1004900079E004C0991F961708F0961B881F7A957B
:1004A000C9F780950895E199FECF1FBA8EBBE09AF7
:1004B00099278DB30895262FE199FECF1CBA1FBA54
:1004C0008EBB2DBB0FB6F894E29AE19A0FBE01964F
:0604D0000895F894FFCF2F
